:020000040000FA
:020000008E2848
:08000800B4000308B5008312E7
:100010000B19192828158B1810280B1919282811C5
:10002000281E1B210C108B1035088300B40E340ED3
:1000300009000B1164002F088500B30AA9080319F1
:100040002428A9030319A814B00803193128300A79
:1000500003193328B10B14282030AF063008B10043
:100060001428AF12031DAF160130B1001428333429
:100070002D344334683461346E346E3465346C34FA
:100080002034523465346C34613479342034433450
:100090006F346E34743472346F346C346C34653451
:1000A0007234203443346F347034793472346934A8
:1000B0006734683474342034283443342934203489
:1000C00050346534743465342034473472346934C0
:1000D00066346634693474346834733420343234AA
:1000E00030343134303420346834743474347034FF
:1000F0003A342F342F3470346934633470347234AA
:100100006F346A3465346334743473342E346F342A
:10011000723467342E3475346B342034831A062AD3
:1001200007309900850183160C308500FF2390006D
:100130006400143081000C14831290018F018E0131
:100140008C01203084008001840A60300406031D85
:10015000A3280130B100FF30AE0081010B110B1656
:100160000B178B168B1790211830B0006E30A9003A
:10017000A810A81CB9280030B000A814C920D220AB
:100180008519B3013308963A031DBE28C921B3016E
:10019000BE28A81C08002818AE1728102009AF0593
:1001A000B0010800281E08002C08AD06031D281207
:1001B000AD002B08AE06031D2812AE00281E080055
:1001C000F720A81AEA280321A81AEA280F21A81A5A
:1001D000EA28F3282818F0282814AF062005AF04D1
:1001E0000C30A900A8100330B00028120800A81293
:1001F00021082C06031D080022082B06031D0800F9
:10020000A81601300800A81223082C06031D0800B8
:1002100024082B06031D0800A81602300800A812A7
:1002200025082C06031D080026082B06031D0800C0
:10023000A816103008002A0803192E29FF3E0319BA
:100240003629FF3E03194229FF3E03194829FF3E84
:1002500003195F29FF3E03196E296A29281D6A299F
:10026000822105196A290130AA0008007421281981
:100270006A29051D6A292B30840040308000023035
:10028000AA0008007421281D6A290330AA0008006A
:100290007B2128196A290230AA00031405190310CA
:1002A000800C031C08002C30840603195B29840091
:1002B00010308000080089210430AA0008002819A5
:1002C0006A290310AB0CAC0CAC0C2C0C1F39AC0025
:1002D0002816702989210530AA00080028196A29E2
:1002E00010100030AA0008001010FC308F00903071
:1002F0008E00101408001010FB308F0064308E0048
:10030000101408001010F5308F0088308E00101483
:1003100008001010D1308F0034308E001014080007
:1003200020308400B60183169B011C141A0880003B
:10033000B6079B0A840A0408283A031D95298312EC
:10034000270836022702031908007830B000851903
:10035000A729C921080020308400A70183169C1812
:10036000AF299B0100089A008312A70783161C156A
:100370008B1355309D00AA309D009C148B179C1840
:10038000BF299B0A840A0408283A031DB229831254
:100390000800EC30AF053D30B0002F14F5212B08DC
:1003A000A2002C08A100AF14F5212B08A4002C08F2
:1003B000A3002F16F5212B08A6002C08A500143049
:1003C000B000851D012A281EE1292812A81CF12948
:1003D000F720A81AAF060321A81AAF060F21A81A02
:1003E000AF060C30A900A810E129281EF529EC3031
:1003F000AF05A8102830281AA9002812A81CFA292D
:1004000008002F081339A000AB21080083128516BD
:040410006400072A53
:02400E008C3FE5
:1042000000000100000001000100010008000C0096
:00000001FF
